:100000000C94D6060C94FE060C94FE060C94FE0688
:100010000C94FE060C94FE060C94FE060C94FE0650
:100020000C94FE060C94FE060C949C1B0C940B1C6A
:100030000C94FE060C94FE060C94FE060C94FE0630
:100040000C94FE060C94FE060C94FE060C94FE0620
:100050000C94FE060C94FE060C94FE060C943D1EB9
:100060000C94FE060C94FE060C94FE060C94FE0600
:100070000C94FE060C94FE060C94FE060C94FE06F0
:100080000C94871E0C94FE060C94FE060C94FE063F
:100090000C94FE060C94FE060C94FE060C94FE06D0
:1000A0000C94FE060C94FE060C94FE06FF048204DB
:1000B000FF201020FF048204FF201020FF04820490
:1000C000FF201020FF048204FF201020FF41204168
:1000D000FF080408FF412041FF080408FF412041B8
:1000E000FF080408FF412041FF080408FF10081022
:1000F000FF824182FF100810FF824182FF1008102A
:10010000FF824182FF100810FF824182FF048204B7
:10011000FF201020FF048204FF201020FF0482042F
:10012000FF201020FF048204FF201020FFFF044165
:1001300082200441FFFF200810042008FFFF044133
:1001400082200441FFFF2008100420080000000066
:10015000FE7F0000FE7FFC3FFE7FFC3FFE7FFC3FFA
:10016000FE7FFC3FFE7FFC3FFE7FFC3FFE7F0000EA
:10017000FE7FFC3FFE7FFC3EFE7FFC3FFE7FFC3FA0
:10018000FE7FFC3FFE7F000000000000000000003A
:1001900000000000C003C003E007E007F00FE00725
:1001A000F00FE007F00FE007F00FE007F00FE007B7
:1001B000F00FE007F00FE007F00FE007E007E007BF
:1001C000C003C003000000000000000001000200A6
:1001D0000400080010002000400080000001000220
:1001E0000004000800100020004000800102040804
:1001F000102040800F00080F0004080C0F000205BB
:10020000080A0D0F00020406080A0C0E0F00010375
:10021000040608090B0C0E0F00010204050608096C
:100220000A0C0D0E0F0001020304050608090A0B53
:100230000C0D0E0F000102030405060708090A0B46
:100240000C0D0E0F0F00000102030405060708083D
:10025000090A0B0C0D0E0F0F000001020304040528
:1002600006070808090A0B0C0C0D0E0F0F00000101
:1002700002020304050506070808090A0A0B0C0D0B
:100280000D0E0F0F0000010202030404050606070D
:100290000808090A0A0B0C0C0D0E0E0F0F000001C6
:1002A00001020303040405060607080809090A0BEE
:1002B0000B0C0C0D0E0E0F0F0000010102020304C7
:1002C000040505060607080809090A0A0B0C0C0DA7
:1002D0000D0E0E0F0F0000010102020303040405BE
:1002E00005060607080809090A0A0B0B0C0C0D0D78
:1002F0000E0E0F0F000001010202030304040505A6
:1003000006060707080809090A0A0B0B0C0C0D0D55
:100310000E0E0F0F0FFFFFFFFFFFD1FFFFF9FFF9D9
:10032000FFC1EBC1FFD3C1E5FFCDF7D9FFCBD5EBC3
:10033000FFFFF9FFFFFFE3DDFFFFDDE3FFEBF7EB7F
:10034000FFF7E3F7FFDFEFFFFFF7F7F7FFFFDFFF51
:10035000FFCFF7F9FFC3DDE1FFDBC1DFFFCDD5D371
:10036000FFDDD5EBFFE1EFC7FFD1D5E5FFC3D5E555
:10037000FFCDF5F9FFC3D5E1FFD3D5E1FFFFEBFFDB
:10038000FFDFEBFFFFF7EBDDFFEBEBEBFFDDEBF769
:10039000FFFDD5F9FFE3DDD3FFC3F5C1FFC3D5E909
:1003A000FFE3DDDDFFC1DDE3FFC3D5D5FFC3F5F519
:1003B000FFE3DDC5FFC1F7C1FFDDC1DDFFEFDDE11B
:1003C000FFC1F7C9FFC1DFDFFFC1FBC1FFC1FDC333
:1003D000FFE3DDE3FFC1F5F3FFE3CDC1FFC3F5C9E3
:1003E000FFDBD5EDFFFDC1FDFFE1DFC1FFE1DFE197
:1003F000FFC1EFC1FFC9F7C9FFF9C7F9FFCDD5D9D3
:10040000FFFFC1DDFFF9F7CFFFFFDDC1FFFBFDFB04
:10041000FFDFDFDFFFFFFDFBFFE7DBC3FFC1DBE744
:10042000FFE7DBDBFFE7DBC1FFE7CBD3FFC3EDFB80
:10043000FFB7ABC7FFC1F7CFFFFFE5DFFFBFCBFFC4
:10044000FFC1F7CBFFFFE1DFFFC3F7C3FFC3FBC76C
:10045000FFE7DBE7FF83DBE7FFE7DB83FFC3F7FBB8
:10046000FFD7D3EBFFE1DBDFFFE3DFC3FFC3DFE356
:10047000FFC3EFC3FFCBF7CBFFF3AFC3FFDBCBD3A0
:10048000FFF7C1DDFFFFC1FFFFDDC1F7FFFBFDFB94
:10049000FFE3EDE3FF0103070F1F3F7FFFFFFEFCBC
:1004A000F8F0E0C080D5F08D14A1C881CFD9F1AFAC
:1004B00020003E004F4646004F4E008040000000A6
:1004C0000000000000000000000000000001FFFF2D
:1004D00082424284FCF8482850F0E02020C0C0400E
:1004E000808000000000000000000000000000000C
:1004F00000000000000000000000000000000000FC
:1005000000000000000000000000000000000000EB
:10051000000000000000000000008080C0C04020FB
:10052000E0E0503048F8F884444482FEFF010000C7
:1005300000000000000000000000000000000000BB
:100540000000000000000000000000000000FFFFAD
:1005500080404080FFFF100810FFFF82C3FFFF08AC
:10056000FF82FFFF01010101010101010101010100
:1005700001FF00000000000000000000000000007B
:10058000000000000000000000FF01010101010166
:100590000101010101010101FF45FF10FFFFC382BD
:1005A000FFFF100810FFFF00808000FFFF00000029
:1005B000000000000000000000000000000000003B
:1005C0000000000000000000000000000000FFFF2D
:1005D00040202040FFFF080408FFFF80C0FFFF0805
:1005E000FF40FFFF000000000000000000000000CE
:1005F00000FF0000000000000000000000000000FC
:10060000000000000000000000FF000000000000EB
:100610000000000000000000FF10FF04FFFF60402A
:10062000FFFF080408FFFF81404081FFFF0000003A
:1006300000000000000000000000000000000000BA
:100640000000000000000000000000000000FFFFAC
:10065000808080807F7F4422243F3F10101F0F0A3C
:100660000F08070704040404040404040404043405
:100670004487403000C0A0A0C000F000F000C020BF
:1006800020C000E0008000E000070404040404042B
:10069000040404040404040407040F090F0F1010D9
:1006A0001F1F2422247F7F40408080FFFF00000026
:1006B000000000000000000000000000000000003A
:1006C0000000000000000000000000000001010127
:1006D000000000000000000000000000000000001A
:1006E00000000000000000000000000000001028D2
:1006F00028CB000808F90A0A00F04B48F300090A61
:10070000FA090801FA01F2090808000000000000D7
:1007100000000000000000000000000000000000D9
:1007200000000000000000000000000000010100C7
:1007300000000000000000000000000000000000B9
:100740000000008080808080808080808080808029
:100750008080808080808080808080808080808099
:100760008080808080808080800000000000010107
:100770000100000000010000000100000100000075
:1007800001000000010000010101000000808080E4
:100790008080808080808080808080808080808059
:1007A0008080808080808080808080808080808049
:1007B00080808080808080000000000000000000B9
:1007C000000000FFFFFFFFFFFFFFFFFFBBB5B5CD40
:1007D000FFFDFD81FDFDFF83EDED83FF81EDED93D9
:1007E000FFFDFD81FDFDFFFFFF0000000000000098
:1007F00000000000000000000000000000000000F9
:1008000000000000000000000000000000FFFFFFEB
:10081000FFFFFFFFFFFFBBB5B5CDFF81FBF781FFFA
:1008200081BDBDC3FFBBFFFFFFFFFFFFFFFFFFFF5A
:10083000FFFFFFFFFFFFFF000000000000000000BF
:100840000000000303030303030303030303030381
:100850000303030303030303030303033B47472B80
:10086000334B7B033F4B03334B7800304848003019
:1008700048300078087878007C48300050582800CC
:1008800000003058500078087000B0C878037B032F
:100890007B0B7303335B5303030303030303030360
:1008A0000303030303030303030303030303030318
:1008B000030303030303030000000000004241435D
:1008C0004B524F4F4D5300454E54455220544845CE
:1008D000000000F090FECFBFFFFFFEF8F8700000B0
:1008E000000000C061F1097F7DFD8DFF30E0000058
:1008F00000700C7303E5340C070D38E302731E7CA3
:10090000002F330046555345003E00484F4D4500EB
:10091000434F4E54494E55450050415553454400B0
:1009200053544154494320464144455300594F557F
:10093000204553434150454400544845204C4947C5
:100940004854532053544159204F4E004954204697
:100950004F554E4420594F550054687265652066C6
:10096000757365732E205468652065786974206FEF
:1009700070656E732E004675736520322F332E001E
:100980004675736520312F332E0041206E6F7465DC
:10099000206D656E74696F6E73207468652074686D
:1009A00069726420646F6F722E0054686520455828
:1009B0004954207369676E207265666C6563747351
:1009C000206E6F206C696768742E00596F75206601
:1009D0006F756E642061206B65792077697468207B
:1009E0006E6F20646F6F722E009F813200000002D4
:1009F000009F812F0000000200D0801F000080496E
:100A00007420686561726420796F752072756E2E2E
:100A100000497420666F756E6420796F752E00AF83
:100A200080100000000400E9801200000003007B39
:100A3000800F00000004008881110000000200DC2B
:100A400080100000000200758011000000010037D6
:100A50008110000000020049800F000000010072B8
:100A6000811000000003002681110000000200C474
:100A7000801300000002002E801100000003008B94
:100A800080130000000100A5801200000004005740
:100A90008011000080546872656520667573657307
:100AA0002072657175697265642E00080B00020280
:100AB00002000009040000010202000005240010E9
:100AC0000105240101010424020605240600010792
:100AD00005810310004009040100020A000000071C
:100AE00005020240000007058302400000040309DC
:100AF0000412010002EF020140412336800001018F
:100B000002030141726475696E6F204C4C430041D1
:100B1000726475696E6F204C656F6E6172646F00F0
:100B200054687265652066757365732072657175AA
:100B3000697265642E00444F204E4F5420464F4C3E
:100B40004C4F5720544845204C49474854532E0099
:100B50005468652066616C736520646F6F722073E2
:100B60007461797320736875742E0020010700008A
:100B7000001500E9000700000007005601150000FD
:100B800000320085011D00000040000B021500002E
:100B9000003200870324000000400087032B000080
:100BA000004000B20332000080000006000C00127A
:100BB0000019001F0025002B00310038003E0044C2
:100BC000004A00500056005C00610067006D007331
:100BD0000078007E00830088008E00930098009DBE
:100BE00000A200A700AB00B000B500B900BD00C175
:100BF00000C500C900CD00D100D400D800DB00DE64
:100C000000E100E400E700EA00EC00EE00F100F390
:100C100000F400F600F800F900FB00FC00FD00FE07
:100C200000FE00FF00FF00FF00FF00FF00FF00FFCD
:100C300000FE00FE00FD00FC00FB00F900F800F6DD
:100C400000F400F300F100EE00EC00EA00E700E43D
:100C500000E100DE00DB00D800D400D100CD00C9E7
:100C600000C500C100BD00B900B500B000AB00A7D1
:100C700000A2009D00980093008E00880083007EF3
:100C800000780073006D00670061005C0056005042
:100C9000004A0044003E00380031002B0025001FB0
:100CA00000190012000C0006000000FAFFF4FFEE2D
:100CB000FFE7FFE1FFDBFFD5FFCFFFC8FFC2FFBCAF
:100CC000FFB6FFB0FFAAFFA4FF9FFF99FF93FF8D20
:100CD000FF88FF82FF7DFF78FF72FF6DFF68FF6373
:100CE000FF5EFF59FF55FF50FF4BFF47FF43FF3F9C
:100CF000FF3BFF37FF33FF2FFF2CFF28FF25FF228D
:100D0000FF1FFF1CFF19FF16FF14FF12FF0FFF0D3F
:100D1000FF0CFF0AFF08FF07FF05FF04FF03FF02A8
:100D2000FF02FF01FF01FF01FF01FF01FF01FF01C2
:100D3000FF02FF02FF03FF04FF05FF07FF08FF0A92
:100D4000FF0CFF0DFF0FFF12FF14FF16FF19FF1C12
:100D5000FF1FFF22FF25FF28FF2CFF2FFF33FF3748
:100D6000FF3BFF3FFF43FF47FF4BFF50FF55FF593E
:100D7000FF5EFF63FF68FF6DFF72FF78FF7DFF82FC
:100D8000FF88FF8DFF93FF99FF9FFFA4FFAAFFB08D
:100D9000FFB6FFBCFFC2FFC8FFCFFFD5FFDBFFE1FF
:100DA000FFE7FFEEFFF4FFFAFF00E81E11241FBE6D
:100DB000CFEFDAE0DEBFCDBF11E0A0E0B1E0E6E9C1
:100DC000FBE502C005900D92AA32B107D9F729E0E0
:100DD000AAE2B1E001C01D92A733B207E1F716E025
:100DE000C6EDD6E004C02197FE010E94C32DC53D8B
:100DF000D107C9F70E940D1F0C94C92D0C94000057
:100E000080913E04089580E0EEE9F4E081118FEFD7
:100E1000002481938193819381930394D1F7089562
:100E2000FC0180918004882311F13FB7F89482E09F
:100E30008093E9002091F200822F90E018161906A5
:100E400014F481E090E0882339F0289844E6409338
:100E50007F044091F1004083222339F02091F20079
:100E6000211103C02BE62093E8003FBF08958FEFC8
:100E70009FEF08952FB7F89483E08093E900909155
:100E8000E800892F807295FF04C09091F20080E401
:100E9000891B2FBF08958091770481110DC082E0D6
:100EA0008093730484E0809374041092760410920B
:100EB000750481E08093770483E794E00895CF93ED
:100EC000DF931F92CDB7DEB76983DC01ED91FC9112
:100ED0000280F381E02D41E050E0BE016F5F7F4F63
:100EE00009950F90DF91CF91089583E08093E900F9
:100EF0008091F200882319F08AE38093E800089536
:100F00000E943A0790E00895CF93DF931F92CDB7E8
:100F1000DEB7FC018485958597FD08C02FEF3FEF74
:100F2000358724870F90DF91CF910895CE010196E8
:100F30000E941007019719F4898190E0F3CF8FEF99
:100F40009FEFF0CF0F931F93CF93DF931F92CDB7F7
:100F5000DEB78C01FC018485958597FF0BC0CE011F
:100F600001960E941007019771F4898190E0F801C1
:100F700095878487F801848595850F90DF91CF91BF
:100F80001F910F9108958FEF9FEFF1CFFC018485A2
:100F9000958597FD0BC09FB7F89482E08093E90098
:100FA0008091F2009FBF90E0019608959FB7F8945A
:100FB00082E08093E9008091F2009FBF90E0089565
:100FC00040916D0450916E0420916B0430916C043B
:100FD00042175307B4F49091E8009570E1F39091B3
:100FE000E80092FD19C08093F10080916D0490910A
:100FF0006E0401968F739927892B19F48EEF8093D5
:10100000E80080916D0490916E04019690936E04B7
:1010100080936D0481E0089580E00895EF92FF923F
:101020000F931F93CF93DF93F82E192FE62E042FE3
:1010300081E0860F880F0E94E00783E00E94E007AE
:10104000CF2DD12FEC0EFD2EF11CCE15DF05B9F002
:1010500007FF13C0FE0184910E94E007182F80E073
:101060000E94E007812321968111EFCFDF91CF917C
:101070001F910F91FF90EF9008958881EDCF81E04F
:10108000F5CFDF92EF92FF920F931F93CF93DF93F1
:10109000D82E8A01EB017B01E40EF51ECE15DF058B
:1010A00059F0D7FE12C0FE0184910E94E0072196FC
:1010B0008111F4CF0FEF1FEFC801DF91CF911F9186
:1010C0000F91FF90EF90DF9008958881EECF0F93FE
:1010D0001F93CF93DF931F92CDB7DEB782E0898352
:1010E00042E450E06BEA7AE080E80E9441080E9406
:1010F0004B07DC0112960D911C910115110589F029
:10110000D801ED91FC910280F381E02DBE016F5F6B
:101110007F4FC801099597FD04C0F801008511852E
:10112000ECCF89810F90DF91CF911F910F9108959E
:10113000615030F02091F100FC0120830196F8CF3E
:10114000289884E680937F0408953FB7F8948091AF
:10115000670490916804A0916904B0916A0426B56F
:10116000A89B05C02F3F19F00196A11DB11D3FBFDF
:10117000BA2FA92F982F8827BC01CD01620F711DAE
:10118000811D911D42E0660F771F881F991F4A95A8
:10119000D1F708958F929F92AF92BF92CF92DF9234
:1011A000EF92FF926B017C010E94A5084B015C014C
:1011B000C114D104E104F104B9F00E94A508681932
:1011C00079098A099B09683E73408105910580F37E
:1011D00021E0C21AD108E108F10888EE880E83E008
:1011E000981EA11CB11CE4CFFF90EF90DF90CF9030
:1011F000BF90AF909F908F9008958F929F92AF92E3
:10120000BF92CF92DF92EF92FF920F931F93CF93F3
:10121000DF936C017B018A0180910F01882309F41F
:101220005CC080918004882309F457C080917204C7
:1012300080FF05C08091E00082608093E000E801BB
:10124000B12C8AEFA82E93E0892E2AE3922E2097C4
:1012500011F4BB20D9F10E943A0781110AC0AA9467
:10126000AA20D9F161E070E080E090E00E94CA0815
:10127000EECF8C171D0611F00CF08C2F9FB7F89451
:101280008092E9002091E80025FD02C09FBFDFCFDA
:10129000282F30E0C21BD30BF701815020F0419181
:1012A0004093F100FACFE20EF31EBB2021F09092A2
:1012B000E800B12CEBCF8091E80085FDE7CF90925C
:1012C000E800BB24B394209709F3F3CF5D9884E63C
:1012D00080937104101611063CF081E090E0F60155
:1012E0009383828310E000E0C801DF91CF911F91CA
:1012F0000F91FF90EF90DF90CF90BF90AF909F90B5
:101300008F90089520912803E0912603F091270300
:10131000CF0102969093270380932603222319F08E
:10132000859194910895808191810895E1E7F0E09D
:1013300080818D7F8083109291004698479810920B
:1013400038040895CF92DF92EF92FF92CF93DF930C
:101350000E948209811520E8920741F4DF91CF9124
:10136000FF90EF90DF90CF900C94960921E02093AE
:101370003804813020E8920751F480912403909141
:10138000250390932703809326030E94820997FDEB
:1013900005C020912303222309F45BC0209122037E
:1013A000211157C021E020932903EC01DF7720971A
:1013B00009F052C081E080932A0346983FE9C32E8A
:1013C0003FE0D32EE12CF12CCAEFD0E0E0913509BB
:1013D000F09136090995811103C081E080932A03B9
:1013E00080912903882329F080912A03882309F416
:1013F00046C047980E948209009709F444C09C01A6
:10140000DE010E947D2DDC01CB0129E0B595A79579
:10141000979587952A95D1F7109290002AE020930E
:101420009100D0929900C092980080932B039093E2
:101430002C03A0932D03B0932E0380917100826042
:1014400080937100DF91CF91FF90EF90DF90CF906C
:10145000089510922903A9CF9E0150E040E060E476
:1014600072E48FE090E00E943C2D69017A0181E0F6
:10147000C81AD108E108F10810922A03A7CF4699AB
:10148000B8CF479AB7CF8FEF9FEFDC01C5CF9C0154
:10149000E1E7F0E090819D7F908381E080932803D5
:1014A00030932703209326033093250320932403AE
:1014B0000C94A209BC0190E080E00C94CA08109240
:1014C0003E043E983F9808953E9A3F9A81E080936B
:1014D0003E040895282F9FB19095907F669B986059
:1014E0001C9B9460922381E0921380E008958038E1
:1014F0009105BCF460347105A4F420E191E061FD34
:1015000094E060FD990F62FD9295687F269FD0015F
:101510001124A80FA256BB4F8C91442319F0892B9C
:101520008C93089590958923FBCF46170CF450C0F7
:1015300047FD4EC060340CF04BC090E082569B4F8C
:10154000E62F67FDE0E040340CF04FE330E1E302CA
:10155000D0011124A078B370A80FB91FF0E14F0299
:10156000B001112460787370860F971FE770F0E068
:10157000E356FB4F477050E04B565B4F6C91A817FA
:10158000B90761F48491FA014491E42FE8233E2FD6
:1015900030953623E223E32BEC930895E4913E2F1C
:1015A00030953623E223E32BEC93A058BF4F8A17E4
:1015B0009B0711F02C93F9CFDC01FA019491892F4C
:1015C00080954C918423E92FE223282F2E2B2C93F6
:1015D0000895CF9388E00E946A0AC0E1811101C09A
:1015E000C0E084E00E946A0A8111C06280E80E9423
:1015F0006A0A8111C46080E10E946A0A8111C86090
:1016000080E20E946A0A8111C16080E40E946A0A35
:101610008111C2608C2FCF9108958432D8F46C313F
:10162000C8F4E82FF0E094E2699FE00DF11D112469
:10163000F595E795E65DFE4F908180FF08C09F70AD
:1016400080E1489FA0011124942B90830895907FFE
:10165000492B40830895843298F46C3188F4282F04
:1016600030E084E2689F200D311D1124F901F595C9
:10167000E795E65DFE4F808120FD82958F7008958D
:101680008DE00895282F30E084E2689F200D311D01
:101690001124F901F595E795E65DFE4F808120FD67
:1016A00082958F7008950E942B0B91E08D3008F485
:1016B00090E0892F08952F923F924F925F926F9200
:1016C0007F928F929F92AF92BF92CF92DF92EF92D2
:1016D000FF920F931F93CF93DF937C016B018A01DD
:1016E000E90197FF02C081509F4F892E992E990CD6
:1016F0009908C80117FF02C081509F4F292E392E2B
:10170000330C33088214930409F45FC082149304E9
:101710000CF0DFC054018FEFA81AB80ABA2CAA2423
:10172000AE18BF0844244394512CBE016C197D09A6
:10173000072E000C880B990B982F872F762F662782
:1017400098012E193F0937FF03C0319521953109C2
:10175000032E000C440B550B0E943C2D66246A940A
:101760007FE7772E211580E838074105510554F4AD
:101770003901213030484F4F5F4F24F46624639481
:1017800060E8762E9301D5010E94B42D20E031E06F
:1017900040E050E00E943C2D5601A20EB31E840C86
:1017A000951C240C351CC501B7FE02C081509F4F0B
:1017B000A60CB71C692F882D0E94530B81119DC068
:1017C000840C951C2814390471F7C601D7FE02C099
:1017D00081509F4FA92EB92EBB0CBB08CE01D7FF5D
:1017E00002C081509F4F492E592E550C5508A41404
:1017F000B50409F45AC0A414B5040CF074C0350142
:101800008FEF681A780A762C66246C187D08882475
:101810008394912CB8016E197F09072E000C880B58
:10182000990B982F872F762F66279E012C193D093B
:1018300037FF03C0319521953109032E000C440B6D
:10184000550B0E943C2DCFEFDFE7211580E83807CC
:101850004105510544F4E901213030484F4F5F4FB5
:1018600014F4C1E0D0E89E01D3010E94B42D20E021
:1018700031E040E050E00E943C2DE20EF31EA80C47
:10188000B91C480C591CC701F7FE02C081509F4F7C
:10189000EC0EFD1E6A2D892F0E94530B81112DC065
:1018A000A80CB91C4A145B0471F781E0DF91CF9159
:1018B0001F910F91FF90EF90DF90CF90BF90AF906E
:1018C0009F908F907F906F905F904F903F902F9060
:1018D0000895C70160E071E00E94A02D5C014424DE
:1018E0004A94542C22CFC60160E071E00E94A02DE2
:1018F0003C0188248A94982C8DCF80E0D7CF90919A
:101900005A04981731F080935A0410925904109297
:1019100058040895672F892F0E942B0B91E089307E
:1019200008F490E0892F0895CF92DF92EF92FF9212
:101930000F931F93CF93DF938C01EB016B0188E42E
:10194000C81AD108780188E4E81AF108B601C7017D
:101950000E948A0C81111CC0085B1F4FB601C80190
:101960000E948A0C811114C0C85BDF4FBE01C80100
:101970000E948A0C81110CC0BE01C701DF91CF917A
:101980001F910F91FF90EF90DF90CF900C948A0CF5
:10199000DF91CF911F910F91FF90EF90DF90CF904B
:1019A0000895DC01605284E0689FB00111246B5EF1
:1019B0007C4FFB01849184278C933196E491E4273A
:1019C0001196EC931197FB013296E491E42712965D
:1019D000EC931297FB013396E491E4271396EC9372
:1019E0000895EF92FF921F93CF93DF93122F1195DB
:1019F00020E8629FE0011124C40FD11DC256DB4FC5
:101A00007C01F7016491FFEFEF1AFF0A662331F0C2
:101A1000412FCE010E94D10C2496F3CFDF91CF91BC
:101A20001F91FF90EF900895809100019091010126
:101A30009C013695322F222737952795282739275D
:101A4000C901892F9927869528273927922F88271A
:101A500082279327909301018093000108952F928C
:101A60003F924F925F926F927F928F929F92AF922E
:101A7000BF92CF92DF92EF92FF920F931F93CF937B
:101A8000DF93CDB7DEB72C970FB6F894DEBF0FBE4D
:101A9000CDBF982E6C87842E722E102FEB8255248A
:101AA0005A94580E81E0890D8983A92CB12C462EB9
:101AB0004A94962F9F5F9A83C62ED12C112341F012
:101AC0009B81992329F040E0692F812F0E940D0B03
:101AD00088E0881508F45EC1871508F4B7C11B8635
:101AE00081E09C85923008F480E09B8580FB94F92E
:101AF0009B8781E0891508F080E09B8580FB97F942
:101B00009B87E92CF12C882D90E09E838D836C01BE
:101B1000CE0CDF1C81E092E2C916D1040CF080E00B
:101B20009B8580FB95F99B878C85082F10E0872D7E
:101B300090E098878F835C01A00EB11E81E09AE14E
:101B4000A916B1040CF080E09B8580FB96F99B8779
:101B50008C858250898344244A94490C682F842DB3
:101B60000E94420B682C690C882349F06981862DFC
:101B70000E94420B882319F09B859F7E9B873C84A3
:101B80003A948EEF890D8A83632D0E94420B5C8408
:101B9000570C882349F0652D8A810E94420B8823C7
:101BA00019F09B859F779B8781E0860D8C83632D41
:101BB0000E94420B882359F06C856F5F670D862D5C
:101BC0000E94420B882319F09B859F7D9B8781E0B3
:101BD000850D8B83682F842D0E94420B882349F04A
:101BE0006B81862D0E94420B882319F09B859F7B79
:101BF0009B876981842D0E94420B81110AC0632D4D
:101C00008A810E94420B811104C08B858F7E8F7761
:101C10008B876981862D0E94420B81110AC0632D3A
:101C20008C810E94420B811104C09B859F7E9F7D09
:101C30009B876B81862D0E94420B81110AC0652D06
:101C40008C810E94420B811104C08B858F7B8F7D1C
:101C50008B876B81842D0E94420B81110AC0652DF8
:101C60008A810E94420B811104C09B859F7B9F77D4
:101C70009B87632D892D0E94420B882349F0632D99
:101C80008FEF860D0E94420B22242394811101C004
:101C9000212C6C85862D0E94420B882349F06FEF22
:101CA000650D862D0E94420B91E09987811101C03C
:101CB0001986652D892D0E94420B882349F0652DD8
:101CC0008FEF860D0E94420B91E09A87811101C02F
:101CD0001A866C85842D0E94420B882341F06FEF99
:101CE000650D842D0E94420B91E0811101C090E0AE
:101CF000211005C08B858F7E8F7D8F778B8789859F
:101D0000811105C08B858F7E8F7D8F7B8B878A8528
:101D1000811105C08B858F7D8F7B8F778B8791118C
:101D200005C09B859F7E9F7B9F779B87EC14FD045E
:101D30000CF0FCC02E2C632D8E2D0E94420B8111C5
:101D400003C08B8581608B87652D822D0E94420B9D
:101D5000811103C09B8594609B878C85823048F0FD
:101D60006981822D0E94420B882319F09B859F7EFA
:101D70009B878AE1A816B1044CF46B81822D0E94E6
:101D8000420B882319F09B859F7B9B878FEFE81A76
:101D9000F80ACCCF871408F459C00FEF882D86506D
:101DA000990B1C019C85970D9B830E94140DB1011A
:101DB0000E948C2D93E0F92EF80E015009F48FCE7D
:101DC0001F2D190D642D812F0E94420B882369F36A
:101DD0006B81812F0E94420B882339F3EE24EA9411
:101DE000E10E642D8E2D0E94420B8823F1F26B814F
:101DF0008E2D0E94420B8823C1F266246394610EEB
:101E0000642D862D0E94420B882379F26B81862DEA
:101E10000E94420B882349F20E94140D272C312C7A
:101E2000B101625071090E948C2D9A81980F9B8399
:101E30000C852C0C3D1C021513040CF06CC04DE0FD
:101E4000602F812F0E940D0B0F5FF5CFEE24EA94D7
:101E5000872D8650990B8C01282C290C0E94140D7B
:101E6000B8010E948C2D23E0F22EF80EEA94EE20A9
:101E700009F435CE9C859F0D9B83692F852D0E948B
:101E8000420B882359F36B81822D0E94420B8823D9
:101E900029F36B806A94662D852D0E94420B88235E
:101EA000E9F2662D822D0E94420B8823B9F26B80E5
:101EB0006394662D852D0E94420B882379F2662D4E
:101EC000822D0E94420B882349F20E94140D282C77
:101ED000312CB101625071090E948C2D1981180FAB
:101EE000092D2A0C3B1C021513043CF44DE06B81B8
:101EF000802F0E940D0B0F5FF6CF2FEF270D2F19AC
:101F0000EB80012F482D662D892D0E942F0D7F2CEF
:101F1000F82C8F2CD3CD4FEF480D4F19EB80012FAC
:101F2000272D6C85862D0E942F0DF3CF0A151B05DA
:101F30007CF5F02E602F842D0E94420B811103C08E
:101F40009B8598609B876F2D862D0E94420B811187
:101F500003C08B8582608B8791E0991548F46F2DC3
:101F60008A810E94420B882319F08B858F778B879B
:101F700092E2C916D1044CF46F2D8C810E94420B61
:101F8000882319F08B858F7D8B870F5F1F4FCECFF6
:101F90009B8595FB112710F996FB002700F997FB0D
:101FA000FF24F0F894FF08C00E94140D64E670E06E
:101FB0000E948C2D869780F1FF2041F00E94140D25
:101FC00064E670E00E948C2D8697B0F1002341F00A
:101FD0000E94140D64E670E00E948C2D8697E0F15B
:101FE000112309F449C00E94140D64E670E00E94B8
:101FF0008C2D869708F040C010E000E08F81988516
:1020000008171907CCF56C85600F40E0862D0E94FB
:102010000D0B0F5F1F4FF2CF10E000E08D819E810E
:10202000081719074CF540E0632D892D800F0E9499
:102030000D0B0F5F1F4FF2CF10E000E08F819885EE
:1020400008171907CCF46C85600F40E0842D0E94BE
:102050000D0B0F5F1F4FF2CF10E000E08D819E81CE
:10206000081719074CF440E0652D892D800F0E9458
:102070000D0B0F5F1F4FF2CF871037C096E09815FA
:10208000A0F58C858F5F898393944DE0682F892D0F
:102090000E940D0B6A946A944DE06981862D0E941E
:1020A0000D0B5A945A944DE0652D862D0E940D0B10
:1020B0004DE0652D892D2C960FB6F894DEBF0FBE2E
:1020C000CDBFDF91CF911F910F91FF90EF90DF90E7
:1020D000CF90BF90AF909F908F907F906F905F90C8
:1020E0004F903F902F900C940D0B2C960FB6F894B8
:1020F000DEBF0FBECDBFDF91CF911F910F91FF903B
:10210000EF90DF90CF90BF90AF909F908F907F9097
:102110006F905F904F903F902F9008958038910579
:1021200014F08FE790E097FF02C090E080E08D5CB4
:102130009C4FFC01808108952F923F924F925F92B5
:102140006F927F928F929F92AF92BF92CF92DF92C7
:10215000EF92FF920F931F93CF93DF93CDB7DEB72C
:102160006C970FB6F894DEBF0FBECDBF5C01322F67
:10217000330F8E2D90E09F838E83A22FA150BB0B37
:10218000CD0102C095958795EA94E2F7889FF0010A
:10219000899FF00DF00D1124CF018C509E4F9B872D
:1021A0008A87862F880F880B962F91958923E32F96
:1021B000F0E0DF01A60FB11D67FDBA95A138B105AA
:1021C0000CF4E2C050E8561B5C8F242F2195942F0D
:1021D000990F990B29232F87E40FF11D47FDFA95DD
:1021E000E134F10514F030E4341B67FD60E0D12CDC
:1021F000AA27BB27AC19BD09BE87AD8747FD40E0C4
:10220000B0E14B02F0011124DF01A078B370B98B6B
:10221000A88B712C612C90E01B8E1A8ED12CC12CB6
:10222000512C412CF12CE12C681B6A8B682F70E03B
:102230007C8B6B8BAC8DA250BB0BBE8BAD8B632F9D
:102240006250770B788F6F8B21E0240F7F85271BDF
:10225000298FAA89A80FBC8D8B1708F0FAC00A2E07
:10226000000CBB0BFD01ED54FC4F208151E0588761
:10227000201708F01886201708F0E5C0EB89FC89C4
:10228000E60DF71D6D897E89E617F7070CF47EC011
:10229000992309F4DEC0B7016C217D217C836B8317
:1022A00070E060E0312C212C142F1770C888D98879
:1022B000AC0DBD1DA256BB4F2C91E12FF0E0E451B7
:1022C000FE4F9491DF84ED2CF12C1986812CF0E0E7
:1022D0001A82912CEC86E31608F0AEC091109F2E66
:1022E000CF88D88CEC14FD040CF092C0F7010E805E
:1022F00002C0F595E7950A94E2F7CA84DB84EC0DF9
:10230000FD1DE491F0E0EE0FFF1FE453FE4FC5907A
:10231000D490EB81FC81EC21FD2151E05D83EF2B1A
:1023200009F41D82E1E0E983F201EC21FD21EF2BAC
:1023300009F41982EA8DFB8DCE22DF22E1E0CD285F
:1023400009F4E0E0CA80CC2009F466C0882009F4D2
:102350006FC0292B1F5F990F183059F42C93998D5A
:10236000CC849C0D903414F4A058BF4F2C9191E074
:1023700010E05FEFE51AF50AFD81F987F82D8E2E42
:102380009A80C980CA82A6CF3C8F1FCF0E8002C020
:10239000F595E7950A94E2F76A857B85E60FF71FC6
:1023A000649170E0660F771F660F771FF501E60FE7
:1023B000F71F9923B9F025903490FB013296EA0D6E
:1023C000FB1D65917491ED85FE856E277F27F101D8
:1023D000E623F723EC20FD206F01CE28DF28DC82E6
:1023E000CB8262CF45905490FB013296EA0DFB1DE3
:1023F000E590F4906D857E856E257F257B8F6A8FB5
:10240000642175217C836B836A8D7B8D12014CCF97
:102410001D82E0E0198296CFD984D11009C09110B5
:1024200007C05981552309F495CFEE2309F492CFC3
:10243000F92FF0952F238ECF2C93CA8CDB8C7B8FBA
:102440006A8F720121018F5F2FEF621A720A9885DD
:1024500000CF6C960FB6F894DEBF0FBECDBFDF91F4
:10246000CF911F910F91FF90EF90DF90CF90BF9091
:10247000AF909F908F907F906F905F904F903F9024
:102480002F9008952F923F924F925F926F927F927A
:102490008F929F92AF92BF92CF92DF92EF92FF9274
:1024A0000F931F93CF93DF9300D000D0CDB7DEB74B
:1024B0007B014A013C832B83302E21E0202E2226F3
:1024C000CB80DC80C61AD70AD7FE03C0D194C19452
:1024D000D1085401A81AB90AB7FE03C0B194A19457
:1024E000B108AC14BD045CF03B812C819C828B82D2
:1024F000832E922E3E2D2F2D7C01832F922F2B8108
:102500003C812E153F055CF0382D292D4C01832F81
:10251000922F3B812C81FC82EB82E32EF22E27014D
:102520004B815C81441A550A3C016818790877FE92
:1025300003C0719461947108820157FE02C00F5F5D
:102540001F4F15950795881699060CF044C081E039
:10255000282F880F330B3A8329834B815C81E41643
:10256000F5060CF48FC0AC14BD040CF04EC050E85E
:1025700085169104F8F48B819C8180349105D0F408
:10258000C4010E948E10082E000C990BF401ED542A
:10259000FC4F208130E0332001F1AC01421B530B92
:1025A0009A014B815C814217530724F4089748171E
:1025B0005907F4F00619170917FF06C089819A8197
:1025C000880E991E040D151D2B813C812F5F3F4FF6
:1025D0003C832B83C2CF8FEFBBCF280F391F4B819A
:1025E0005C812417350734F708968417950714F78C
:1025F000F401ED5CFC4F80816B816052680F70E0EC
:10260000422DC4010E94770AD5CF8B819C818038EE
:10261000910580F690E48916910460F68B819C8187
:102620000E948E10082E000C990BEB81FC81ED545A
:10263000FC4F208130E03320C9F0AC01421B530B2A
:10264000841695060CF0B6CF0897881699060CF0FC
:10265000B1CFEB81FC81ED5CFC4F808160EE680DB9
:10266000680F70E0422D8B819C81CCCF280F391FE1
:10267000281539050CF09ECF0896881599050CF0A1
:1026800099CFE7CF0F900F900F900F90DF91CF91E0
:102690001F910F91FF90EF90DF90CF90BF90AF9080
:1026A0009F908F907F906F905F904F903F902F9072
:1026B00008958F929F92AF92BF92CF92DF92EF9246
:1026C000FF920F931F93CF93DF938901AFE3B4E0A1
:1026D0002D913C9111977C01E21AF30A12968D918B
:1026E0009C911397FB01E81BF90B1596CD91DC919A
:1026F00016971796CD90DC909E01D7010E94B42DBD
:10270000872E982EA92EBB24A7FCBA949601DF0130
:102710000E94B42D672F782F892F992787FD9A95CE
:10272000861A970AD8018D929C92D7010E94B42DE7
:10273000C72ED82EE92EFF24E7FCFA949E01DF0174
:102740000E94B42D672F782F892F992787FD9A959E
:10275000C60ED71EFA01D182C082DF91CF911F91A0
:102760000F91FF90EF90DF90CF90BF90AF909F9030
:102770008F900895CF92DF92EF92FF920F931F9365
:10278000CF93DF9300D000D0CDB7DEB77A016901D7
:102790009E012D5F3F4FAE014F5F5F4F0E94591367
:1027A0000B811C81003211056CF0A981BA81B7FF41
:1027B0000BC088279927801B910B880F991FA8179A
:1027C000B90754F480E026C0109731F0C801880F93
:1027D000991F8A179B07B4F321E430E00E94BC2DB7
:1027E0009801012E000C440B550B0E943C2DF70163
:1027F0003183208380E890E2B8010E94A02DF60189
:1028000071836083F70180819181805C9F4F918308
:10281000808381E00F900F900F900F90DF91CF9108
:102820001F910F91FF90EF90DF90CF900895AF929E
:10283000BF92CF92DF92EF92FF920F931F93CF93AD
:10284000DF9300D000D0CDB7DEB76C01CB01BA0169
:10285000122F9E012F5F3F4FAE014D5F5F4F0E94D1
:10286000BA13882309F4A5C0A980BA801A9D700103
:102870001B9DF00C1124F7FE03C02FE7E20EF11CA4
:10288000EE0CEF2CEE1CFF081B81812F9C810E9417
:102890008E10013009F454C09E2D990F4A2D491B0A
:1028A000840F312F3E19632F032E000C770BA701E5
:1028B0005527519541955109440F551F64177507C8
:1028C0000CF477C0A3942091D608EEE9F8E050E02C
:1028D00040E0942F4217B0F19091D608983008F458
:1028E00099C0492F4150550BBA0127E0249FF001B0
:1028F000259FF00D1124E256F74F26812A1508F086
:1029000058C020E017E0422F50E0461757070CF060
:1029100086C0149FD001159FB00D1124A256B74F49
:102920004F5F5F4F149FF001159FF00D1124E25689
:10293000F74F412F01900D924A95E1F72F5FE3CFBA
:102940008E19AFCFBA01A6814F5F5F4F3796AA1697
:1029500008F0BFCF2830E0F541E0420F4093D608A1
:1029600057E0259FD0011124A256B74FAD01475023
:10297000510967E0FA0101900D926A95E1F7215043
:10298000DA01921798F3983009F4A6CF57E0959F93
:10299000F0011124DF01A056B74F9C91E256F74F8A
:1029A000D182C08233838483E582A6829E7F9D7F0D
:1029B0009C930F900F900F900F90DF91CF911F91EC
:1029C0000F91FF90EF90DF90CF90BF90AF90089560
:1029D000992379F320E06150710917E0422F50E00C
:1029E00046175707E4F4149FD001159FB00D11242A
:1029F000A256B74F4F5F5F4F149FF001159FF00D28
:102A00001124E256F74F412F01900D924A95E1F7BC
:102A10002F5FE4CF21E0290F2093D608B7CF915044
:102A2000B5CFAF92BF92CF92DF92EF92FF920F930A
:102A30001F93CF93DF93CDB7DEB728970FB6F894E7
:102A4000DEBF0FBECDBF8A0179019E012D5F3F4FD2
:102A5000AE014F5F5F4F0E9459139E01295F3F4FA8
:102A6000AE014B5F5F4FB701C8010E9459132B8124
:102A70003C816F817885203231050CF06EC0603268
:102A800071050CF459C009811A814D815E81401B8A
:102A9000510BE0E2F0E0DF01A21BB30B4A9FC00143
:102AA0004B9F900D5A9F900D1124621B730B0E9437
:102AB000A02D600F711F7A836983FC83EB830B81E8
:102AC0001C81EF81F88580E8E82E80E2F82EC701AE
:102AD000BF010E94A02D5B0150E2A50EB11CAD818B
:102AE000BE8121E430E00E94BC2D9F01FF0F440B0A
:102AF000550B0E943C2D69018FE3C80ED11CC70104
:102B0000B8010E94A02D7B0140E2E40EF11CA981D6
:102B1000BA8121E430E00E94BC2D9801110F440BD2
:102B2000550B0E943C2DC901805C9F4F00E0950130
:102B3000A601B7010E94421228960FB6F894DEBF94
:102B40000FBECDBFDF91CF911F910F91FF90EF90FE
:102B5000DF90CF90BF90AF900895603271050CF078
:102B6000AECF0D811E8149815A81401B510BE0E29D
:102B7000F0E0DF01A61BB70B4A9FC0014B9F900DF1
:102B80005A9F900D1124A901461B570BBA010E94B0
:102B9000A02D600F711F7E836D83F887EF838FCF29
:102BA0008F929F92AF92BF92CF92DF92EF92FF925D
:102BB0000F931F93CF93DF93CDB7DEB728970FB650
:102BC000F894DEBF0FBECDBF8A0179019E012D5F53
:102BD0003F4FAE014F5F5F4F0E9459139E01295F27
:102BE0003F4FAE014B5F5F4FB701C8010E945913C1
:102BF0002B813C816F817885203231050CF070C0CB
:102C0000603271050CF459C009811A814D815E81D1
:102C1000401B510BE0E2F0E0DF01A21BB30B4A9F27
:102C2000C0014B9F900D5A9F900D1124621B730B96
:102C30000E94A02D600F711F7A836983FC83EB8350
:102C40000B811C81EF81F88580E8882E80E2982E28
:102C5000C401BF010E94A02D90E2E92EF12C570182
:102C6000A61AB70AAD81BE8121E430E00E94BC2DD6
:102C70009F01FF0F440B550B0E943C2D69018FE310
:102C8000C80ED11CC401B8010E94A02DE61AF70A93
:102C9000A981BA8121E430E00E94BC2D9801110F76
:102CA000440B550B0E943C2DC901805C9F4F01E0F5
:102CB0009501A601B7010E94421228960FB6F8941A
:102CC000DEBF0FBECDBFDF91CF911F910F91FF905F
:102CD000EF90DF90CF90BF90AF909F908F9008952E
:102CE000603271050CF0ACCF0D811E8149815A8193
:102CF000401B510BE0E2F0E0DF01A61BB70B4A9F3F
:102D0000C0014B9F900D5A9F900D1124A901461BA5
:102D1000570BBA010E94A02D600F711F7E836D8337
:102D2000F887EF838DCF2F923F924F925F926F92F1
:102D30007F928F929F92AF92BF92CF92DF92EF924B
:102D4000FF920F931F93CF93DF93CDB7DEB7A69774
:102D50000FB6F894DEBF0FBECDBFCB01BA0149015B
:102D6000EB8EC8A2ABA29E012D5F3F4FAE014F5F1D
:102D70005F4F0E9459139E01295F3F4FAE014B5F89
:102D80005F4FB801C4010E9459132D813E8137FF66
:102D90000BC08F819885919581959109880F991F16
:102DA000281739070CF430C2E981FA81AB80BC8066
:102DB0001E161F063CF4A501440F551F4E175F0752
:102DC0000CF422C26F81788580E2A816B1040CF061
:102DD000E7C0603271050CF417C200E210E0780120
:102DE000EA18FB086B01CA18DB08C701A5E0880FC9
:102DF000991FAA95E1F7B6010E94A02D762E2E1BF1
:102E00003F0B2E9DC0012F9D900D3E9D900D1124D6
:102E1000B6010E94A02DE60FF71FFA83E9831C83F9
:102E20000B83B0E2FB2E1B8E0B811C81A981BA8122
:102E300021E430E00E94BC2D9801012E000C440BCF
:102E4000550B0E943C2D29873A874B875C87CF80A2
:102E5000D884290170E4470E511CAD81BE8121E464
:102E600030E00E94BC2D96010D2C000C440B550B3C
:102E70000E943C2D49018FE3880E911C481459048F
:102E80000CF0C2C1181419040CF0BEC190E8491628
:102E900051040CF0B9C120E830E2C901B8010E9428
:102EA000A02D8B01C901B6010E94A02D6B0157FE18
:102EB00029C080EC9FEF5C01E985FA85AE1ABF0A54
:102EC000140124183508032C000C440855086F2DF4
:102ED0006719770B9B01D5010E94B42DA2019101C6
:102EE0000E943C2D720E9601201B310BD5010E94D1
:102EF000B42DA20191010E943C2D020F131F1B8EC5
:102F0000512C412CC401841995099E878D8797FD0A
:102F10000196FC01F595E795FA87E987F7180C15F6
:102F20001D050CF06DC09601201B310B3D8F2C8FC1
:102F300031E03F8B4A8E9F8E8E8E80E888169104FA
:102F400024F0EFE7F0E0FF8FEE8F29853A853A8B8A
:102F5000298B12016F89062E000C770B7AA369A3C7
:102F60007F8970957CA38F2D90E09EA38DA3F101A6
:102F7000ED5CFC4F608037FC0AC0F101ED54FC4F62
:102F8000FE8BED8B8081801711060CF473C1FA8DD6
:102F9000F215130409F032C1FF5FFA8FD12C8EC0F5
:102FA00050E2F52E712C603271050CF03DCF00E23D
:102FB00010E06801C61AD70AA61AB70A40EEB60191
:102FC0004603C001479F900D1124B5010E94A02D1A
:102FD00070E2F72EF60EE21BF30BEC9DC001ED9DA7
:102FE000900DFC9D900D1124B5010E94A02D260F7F
:102FF000371F3E832D8318870F83712C18A214CF9F
:10300000B8016C197D097D8F6C8F7FEF7F8B92CF1C
:1030100020E0A62C062C000CBB08C62CC01AA0165B
:10302000B1060CF4C12CB501600F711F788B6F874E
:103030006134710524F080E490E0988B8F874F8590
:103040006C2D822D0E94950A0830110514F1872DF0
:103050008F7190E0FC01E455FF4FE490FC01E453D4
:10306000FF4F2491288FFC01E451FF4F3491398F99
:10307000FC01E45FFE4FF490822F8E2183238F2189
:103080008F3F09F058C020E04F856C2D822D0E94A3
:10309000950AED89FE898081811105C080913304F4
:1030A0008F5F809333040F3F110509F00CF4A2C029
:1030B0002FEFED89FE892083DD24D39482149304BD
:1030C00009F4A2C069857A858C8D9D8D681B790B6A
:1030D0007A87698789A19AA1800F911FC62CC81A87
:1030E0007101FF24ECA18E0F801B680E29853A85A3
:1030F00037FFA3C069A17AA1060F171F8D859E8592
:10310000280F391F3A872987DD2091F037FF10C03B
:10311000013211056CF4662D600F70E040E0C701CC
:103120000E94770A6C2D70E040E0C7010E94770A88
:10313000FF89CF1ADBCF888D8E29698D862B8F2949
:1031400009F4A7CFD12CA01AB10AB6016A197B09DC
:1031500090E080E029E0660F771F881F991F2A956D
:10316000D1F75801AA0CBB1C95010B2C000C440B89
:10317000550B0E945B2D3C8B2B8B80E092E0B501C0
:103180000E948C2D5B01672B19F4AA24A394B12C07
:103190007F85C71608F07DCF2B893C8984E0369562
:1031A00027958A95E1F7822F8F718830E8F080317A
:1031B000E8F08831E8F4898D90E0277002C0959599
:1031C00087952A95E2F780FF05C040E0B601C1016E
:1031D0000E94770A8B899C898A0D9B1D9C8B8B8B07
:1031E0009FEFC91AD90AD4CF8E2DE6CF888DE4CFB0
:1031F0008F2DE2CFED89FE8900835ECF2E8D3F8D2E
:10320000221633060CF0CACEA6960FB6F894DEBF8F
:103210000FBECDBFDF91CF911F910F91FF90EF9027
:10322000DF90CF90BF90AF909F908F907F906F90E6
:103230005F904F903F902F900895E989FA892DA1D2
:103240003EA1E21BF30BFA8BE98B69897A8977FF40
:1032500008C073948D859E85680F791F7A8B698B62
:10326000F4CF9FEF291A390AE0E82E1631040CF446
:103270007ECECACFFBA180E0FF2321F0C101809563
:1032800090958170FB8DFF2321F04214530409F4C3
:10329000BFCE28A1222321F08214930409F4B8CED2
:1032A0002FEF882309F4B5CE25E5B3CE2F923F92B8
:1032B0004F925F926F927F928F929F92AF92BF9246
:1032C000CF92DF92EF92FF920F931F93CF93DF93F2
:1032D00000D01F92CDB7DEB7E82EC62E0E942B0B72
:1032E000182F2C2D30E03B832A838E2C912C40917B
:1032F00048045091490480914C04F401E81BF10901
:1033000060914A0470914B0480914D04281B31094F
:103310004E9FC0014F9F900D5E9F900D1124629FA4
:10332000D001639FB00D729FB00D11248A1B9B0BBF
:1033300081159E4F34F1E69FC001E79F900DF69FE7
:10334000900D1124429FB001439F700D529F700D4C
:103350001124860F971F81159E4F9CF0153039F56B
:103360008A819B81982F8827AC0140585F4F782D28
:10337000662760587F4F00E02AE38CE891E00E94C6
:1033800017140F900F900F90DF91CF911F910F9115
:10339000FF90EF90DF90CF90BF90AF909F908F9075
:1033A0007F906F905F904F903F902F9008951430D2
:1033B000A1F4809194042CE581112CE68A819B81F3
:1033C000982F8827AC0140585F4F782D66276058AA
:1033D0007F4F01E08CE491E0D2CF6C2D8E2D0E94C6
:1033E000530B882371F28091330487FDCACF982C48
:1033F00088242A813B81322F22273B832A83340170
:1034000073944A805B8053946C2D8FEF8E0D0E94D5
:10341000530BD82E6C2D81E08E0D0E94530B8983A7
:103420006FEF6C0D8E2D0E94530BF82E61E06C0D2A
:103430008E2D0E94530BB82E212F2150330B1901D2
:1034400025E0220C331C2A95E1F7C101845D9E4FD3
:103450001C01D1102BC080913F049091400488152D
:10346000990524F5B11009C0CC24C394809141047E
:1034700090914204841595050CF0C12CF1100BC0FD
:10348000EE24E39480914104909142042A813B818F
:10349000281739070CF0E12CAA24A3948201940187
:1034A0004A815B81B401C1010E949316B11028C00A
:1034B0008091410490914204481659060CF53981D7
:1034C000311109C0CC24C39480913F0490914004F1
:1034D000861597050CF0C12CD11009C0EE24E39499
:1034E00080913F0490914004881699060CF0E12CDD
:1034F000A12C82019301A201B401C1010E94931683
:10350000898181112BC080913F04909140046816FD
:10351000790624F5F1100BC0CC24C39480914104AA
:10352000909142042A813B81281739070CF0C12C65
:10353000B11009C0EE24E3948091410490914204BB
:10354000841595050CF0E12CAA24A3940A811B8113
:103550009301A201B301C1010E949316F11011CF92
:1035600080914104909142042A813B818217930704
:103570000CF007CFD11009C0CC24C39480913F0434
:1035800090914004881699060CF0C12C39813111B4
:103590000AC0FF24F39480913F0490914004861563
:1035A00097050CF0F12CA12CEF2C0A811B819401C2
:1035B000A801B301C1010E949316E3CEE0E4F0E05C
:1035C000E81BF109FF27EE0FFF1FE755F44F859128
:1035D00094910895CF92DF92EF92FF920F931F93F1
:1035E000CF93DF93C0918404D091850480918804A7
:1035F0000E94DE1AE0918804F0E0EE0FFF1FE7550D
:10360000F44F459154916CE3689F9001699F300D90
:10361000112437FF02C021503F4F832F992787FD88
:103620009A958C0F9D1F97FF02C081509F4F192FB5
:103630008CE3849FE001859FD00D1124D7FF02C049
:10364000C150DF4FCD2FDD0FDD0B809186049091AF
:103650008704C80FD91FD7FF02C0C150DF4F6D2F9D
:10366000812F0E942B0B8A3061F08C3009F451C0FD
:103670008430F1F48091940481111AC080E29BE0BF
:103680004AC04BE06D2F812F0E940D0B8BE69BE013
:103690000E94470A80E59BE0909383048093820414
:1036A0008AE58093810480919A048F5F80939A04C5
:1036B000C0918604D09187046E0180E3C81AD108B6
:1036C0000091840410918504780180E3E81AF108E0
:1036D000B601C7010E948A0C811125C0005D1F4FF1
:1036E000B601C8010E948A0C81111DC0E096BE017E
:1036F000C8010E948A0C811116C0BE01C701DF916A
:10370000CF911F910F91FF90EF90DF90CF900C948D
:103710008A0C86E39BE090938304809382048AE57D
:1037200080938104C5CFDF91CF911F910F91FF90BE
:10373000EF90DF90CF9008951F920F920FB60F92E7
:1037400011248F939F938091E1009091E100937FEA
:103750009093E10083FF0FC01092E90091E09093F5
:10376000EB001092EC0092E39093ED001092800435
:1037700098E09093F00082FF22C093E09093E900DC
:103780009091F200992319F09AE39093E8009091B8
:103790007104992341F090917104915090937104B8
:1037A000911101C05D9A90917F04992341F090910D
:1037B0007F04915090937F04911101C0289A84FF57
:1037C00018C08091E2008E7E81608093E20080913B
:1037D000E1008F7E8093E100809172048E7E806193
:1037E000809372049F918F910F900FBE0F901F9046
:1037F000189580FFF7CF8091E2008E7E80618093E4
:10380000E2008091E1008E7E8093E100809172045D
:103810008E7E8160E5CF1F920F920FB60F9211241A
:10382000CF92DF92EF92FF920F931F932F933F93CC
:103830004F935F936F937F938F939F93AF93BF93B8
:10384000EF93FF93CF93DF93CDB7DEB76C97DEBFD7
:10385000CDBF1092E9008091E80083FF25C068E0A9
:10386000CE0145960E94980882EF8093E8008D89EA
:1038700087FF39C09091E80090FFFCCF982F907699
:1038800009F034C19E894F89588D2F89F88C911188
:1038900031C0803861F5809170048093F1001092FE
:1038A000F1008EEF8093E8006C960FB6F894DEBFBF
:1038B0000FBECDBFDF91CF91FF91EF91BF91AF913F
:1038C0009F918F917F916F915F914F913F912F9138
:1038D0001F910F91FF90EF90DF90CF900F900FBE50
:1038E0000F901F9018959EEF9093E800C7CF10920D
:1038F000F100D5CF913059F48111D3CF413051052A
:1039000081F6809170048D7F80937004CACF9330CC
:1039100049F48111C6CF4130510519F680917004E8
:103920008260F2CF953041F48091E80080FFFCCFB7
:1039300020682093E300B5CF963009F0A9C00B8D25
:103940001C8D22E01092E90010926E0410926D041A
:10395000F2122EC010926C0410926B040E94670841
:103960001F8299E09983FA8291E09E8390EA98877A
:103970009AEF998720916D0430916E04275F3F4F35
:103980003C832B838D831092E90010926E04109279
:103990006D0410936C0400936B0449E050E0BE0189
:1039A0006F5F7F4F80E00E9441080E94670879CFD7
:1039B00010936C0400936B040E944B07DC01129679
:1039C0000D911C910115110509F451C1D801ED911A
:1039D000FC910480F581E02DBE016B5E7F4FC80134
:1039E0000995009709F03EC1F80100851185EACFDD
:1039F000F3E0FF120EC08F89882309F440C08230A3
:103A000061F440E860E18FE09BE00E940E088111C4
:103A100048CF81E28093EB0047CF813029F440E822
:103A20006BE083E09BE0F1CF833099F70E944B0776
:103A3000DC011296ED90FC908E010F5F1F4F680124
:103A4000E114F10479F0D701ED91FC910680F78142
:103A5000E02DB801C7010995080F111DF701E08499
:103A6000F184EECFD8011C92F60101900020E9F715
:103A70003197BF016C197D0940E0C601C6CF6DEEDC
:103A80007AE0FB01449150E080E80E94410809CFB0
:103A9000973009F4BECF983021F481E08093F10093
:103AA00000CF993009F0FDCE837009F0B2CFE1E18B
:103AB000F1E081E031E096E32191222371F08093DF
:103AC000E9003093EB00DF0111972C912093EC007B
:103AD0009093ED008F5F873079F78EE78093EA004F
:103AE0001092EA008F8980938004DBCE8B8D9C8DB1
:103AF0001092E90010926E0410926D0490936C0481
:103B000080936B04898D811192C08E899D89913A31
:103B100049F4813209F07DCF47E050E068E071E080
:103B200080E0B3CF913209F074CF833269F48F898A
:103B3000988DB0E0A0E08093040190930501A093DC
:103B40000601B0930701ADCE803269F48091E800A0
:103B500082FFFCCF67E088E091E00E9498088BEF3D
:103B60008093E8009ECE823209F09BCE8F898093AD
:103B70000F01EEEFFFE7859194918B3F9C4D51F142
:103B8000E0E0F8E08091080190910901A0910A011C
:103B9000B0910B01803B9440A105B105F1F48091F7
:103BA0000F0180FD1AC0EE3F8AE0F80789F587E72C
:103BB00097E7918380838091600080936F0488E110
:103BC0009BE00FB6F894A895809360000FBE909389
:103BD000600067CEEEEFFAE0D5CF80819181873724
:103BE000974709F05ECEA895809160008861809328
:103BF000600080916F0480936000EE3F2AE0F2073E
:103C000089F08091FE0A9091FF0A9183808349CECA
:103C1000808191818737980751F29093FF0A8093B2
:103C2000FE0AC5CF1092FF0A1092FE0A3ACE0E94F9
:103C30004B07DC0112960D911C910115110509F439
:103C4000E8CED801ED91FC910190F081E02DBE010C
:103C50006B5E7F4FC8010995811123CEF801008565
:103C60001185EBCF181619060CF41BCED2CEF1E05D
:103C7000FF12BECE61EF7AE004CF1F920F920FB613
:103C80000F9211242F933F938F939F93AF93BF93E2
:103C90008091630490916404A0916504B0916604DE
:103CA0003091620423E0230F2D3758F50196A11DB2
:103CB000B11D209362048093630490936404A093E5
:103CC0006504B09366048091670490916804A091A4
:103CD0006904B0916A040196A11DB11D8093670427
:103CE00090936804A0936904B0936A04BF91AF9164
:103CF0009F918F913F912F910F900FBE0F901F902A
:103D0000189526E8230F0296A11DB11DD2CF1F9250
:103D10000F920FB60F9211242F933F934F935F93FF
:103D20006F937F938F939F93AF93BF93EF93FF9383
:103D300080912B0390912C03A0912D03B0912E0321
:103D4000892B8A2B8B2B09F440C080912A03811187
:103D50000BC088B190E4892788B980912903882312
:103D600019F088B1805888B980912B0390912C0369
:103D7000A0912D03B0912E03181619061A061B06E2
:103D80009CF480912B0390912C03A0912D03B09172
:103D90002E030197A109B10980932B0390932C0363
:103DA000A0932D03B0932E03FF91EF91BF91AF919C
:103DB0009F918F917F916F915F914F913F912F9143
:103DC0000F900FBE0F901F9018950E94A209ECCF84
:103DD000E7EDF8E01382128288EE93E0A0E0B0E015
:103DE00084839583A683B7838BE191E0918380835D
:103DF0008FEF9FEF9587848780E097E09093360957
:103E00008093350980E090E89093340980933309DA
:103E100046983E9A47983F9A0895CF93DF93CDB73F
:103E2000DEB765970FB6F894DEBF0FBECDBF7894AE
:103E300084B5826084BD84B5816084BD85B58260AF
:103E400085BD85B5816085BD80916E008160809360
:103E50006E001092810080918100826080938100C9
:103E600080918100816080938100809180008160D9
:103E70008093800080919100826080939100809176
:103E80009100816080939100809190008160809387
:103E900090008091C10084608093C1008091C10036
:103EA00082608093C1008091C10081608093C100D5
:103EB0008091C30081608093C3008091C0008260C4
:103EC0008093C0008091C20081608093C200809185
:103ED0007A00846080937A0080917A008260809377
:103EE0007A0080917A00816080937A0080917A00D4
:103EF000806880937A00109280041092700410926F
:103F000072048091D70081608093D70080EA80930B
:103F1000D80089B5806189BD89B5826089BD09B441
:103F200000FEFDCF61E070E080E090E00E94CA08F2
:103F30008091D8008F7C80618093D8008091E000D0
:103F4000807F8093E0008091E1008E7E8093E1008D
:103F50008DE08093E200559A209A81EC80937C005A
:103F600085B1806F85B984B1877E84B984B1876E4D
:103F700084B95E9A5F988AB1806D8AB9769A6E9894
:103F800081B3806F81BB899880B38D7080BB80E5E1
:103F90008CBD81E08DBD85E090E00E945A0A5F9A59
:103FA00085E090E00E945A0A5E985C98E5EAF4E0A9
:103FB00082EB94E024912EBD00000DB407FEFDCFEE
:103FC00031968E179F07B1F75C9A81E88093640061
:103FD0008091650081608093650080E80E946A0A94
:103FE0008823A9F05C9885EA8EBD00000DB407FE19
:103FF000FDCF5C9A2E982F982D9880916400806256
:104000008093640081E083BF889513BEFCCF84E079
:104010000E946A0A882309F446C02D9884E80E9409
:104020006A0A8823D9F02D9A88EC90E00E945A0AF7
:104030002F9882E090E00E94262D8F3F29F06FEFAD
:1040400082E090E00E942E2D84EF91E00E945A0AB7
:104050002F9A84E80E946A0A8111FBCF84E10E94B2
:104060006A0A8823D9F02D9A88EC90E00E945A0AB7
:104070002E9882E090E00E94262D882329F060E0AF
:1040800082E090E00E942E2D84EF91E00E945A0A77
:104090002E9A84E10E946A0A8111FBCF88EC90E09D
:1040A0000E945A0AB4CF2D9A81E28093020190E0D7
:1040B00080E00E94262D813009F09AC00E94640A97
:1040C000809164008E7F8093640080917A00806488
:1040D00080937A0080917A0086FDFCCF0091780071
:1040E000109179000E94A508AB01BC018091640089
:1040F000816080936400C801B0E0A0E0DC019927F2
:104100008827840F951FA61FB71FBC01616070939D
:104110000101609300010E9496091092830410929D
:1041200082041092810410925A0410925404109246
:104130005604109255041092510410929404109257
:104140005304109258042FB7F8948091630490910F
:104150006404A0916504B09166042FBF80935E044F
:1041600090935F04A0936004B0936104D987C887DB
:104170008FB7F89440916304509164046091650492
:10418000709166048FBF80915C0490915D04840FF0
:10419000951F20915E0430915F04821B930B9093D6
:1041A0005D0480935C0440935E0450935F046093CD
:1041B0006004709361048FB7F89440916304509148
:1041C000640460916504709166048FBF809132032E
:1041D000242F281B822F90913103992361F0109294
:1041E000310380E090E0892B19F20E940000C0CFDB
:1041F0000E945F0A65CF90910201291740F48F5FFA
:10420000891778F731E033BF889513BEEACF81E094
:10421000809331034093320380912F0390913003B8
:1042200001969093300380932F0380915A0420913C
:104230005C0430915D04223231050CF463C7909127
:104240005B049F5F90935B048230C1F180F488230C
:1042500009F47FC6813009F4F4C380915C04909125
:104260005D04819790935D0480935C04DECF83307E
:1042700009F4F7C6843089F7809158049091590465
:104280008E31910528F40196909359048093580437
:1042900080915804909159044E9709F027C70E94C5
:1042A000E90A807309F422C7809158049091590457
:1042B00001969093590480935804CFCF0E94E90A45
:1042C000982F9073903369F49091390490739033E0
:1042D00041F0809339040E94960983E00E947F0C8C
:1042E000BCCF8093390480918104882349F08150A8
:1042F00080938104811104C010928304109282047F
:104300000E94E90A982F9170382F327084FF77C08D
:10431000792E7194332319F077247394791A20E05D
:1043200090919004992319F091509093900490915A
:104330008D0492170CF06AC09F5F90938D0490914A
:104340008D04959520918804920F9093880482FBA8
:10435000992490F883FD9A9485FF03C081E0911021
:1043600001C080E080939104911003C0772009F48C
:1043700054C080913704811114C08091560481117A
:1043800010C08091380481110CC089EE99E00E9420
:10439000470A80919104882309F43DC087E0809307
:1043A000370480913704882319F0815080933704B3
:1043B0008091350490913604019690933604809351
:1043C000350480918E04882359F1815080938E04A6
:1043D0000E94140D837099271FEF180F0E94140D6F
:1043E0008F719927805190914E049817E4F49A5F49
:1043F00090934E048917F4F480934E041BC020E080
:1044000091112AEF31112A5F712C8ACF29170CF0F4
:1044100096CF915092CF8AE0C2CF10923704C1CF8D
:1044200010E080E0E0CF89172CF4965090934E0472
:10443000981714F390914F04911744F49D5F909353
:104440004F04191754F410934F0407C019172CF494
:10445000935090934F049117B4F3809188040E9475
:10446000DE1A6C0180918804E82FF0E0EE0FFF1F48
:10447000E755F44FA590B490805C0E94DE1A7C0151
:10448000E0918804E05CF0E0EE0FFF1FE755F44F89
:104490000591149180919104882309F4D6C180E19B
:1044A000E92D990CFF0B882E880F9908AE9EC0014C
:1044B000AF9E900DBE9E900D1124B4010E94A02DC0
:1044C000A0908B04B0908C04A60EB71E272D770CFD
:1044D000330BCE9EC001CF9E900DDE9E900D112419
:1044E000B4010E94A02DE0918904F0918A04E60FA6
:1044F000F71FE29EC001E39E900DF29E900D1124E5
:1045000048E1E42EF12CB7010E94A02DE60FF71F21
:10451000F0938A04E0938904029FC001039F900DE9
:10452000129F900D1124B7010E94A02DA60EB71E58
:10453000B0928C04A0928B04B7FE03C093E0A90E46
:10454000B11CB594A794B594A794F7FD33968F0149
:10455000159507951595079580918404909185048C
:10456000800F911F9093850480938404809186042A
:10457000909187048A0D9B1D9093870480938604F5
:104580000E94EA1A882381F1809186049091870421
:104590008A199B0990938704809386040E94EA1AE3
:1045A000882311F18091840490918504801B910BE4
:1045B000909385048093840480918604909187046D
:1045C0008A0D9B1D90938704809386040E94EA1AAB
:1045D000882351F080918604909187048A199B0961
:1045E00090938704809386042091890430918A04F3
:1045F00047E0429FC001439F900D112497FD07960D
:1046000003E0959587950A95E1F790938A04809346
:10461000890420918B0430918C0447E0429FC001B3
:10462000439F900D112497FD079613E0959587956C
:104630001A95E1F790938C0480938B0480919304F6
:10464000843638F490919004911103C08F5F809369
:10465000930480918F04882319F0815080938F04F4
:10466000809184049091850497FF02C081509F4FF0
:10467000F92E009186041091870417FF02C00150A3
:104680001F4F612F8F2D0E942B0B863009F425C1FF
:1046900008F0DDC0853009F4F8C0E0908604F090A1
:1046A0008704009184041091850480915404882328
:1046B00009F476C1C0903A04D0903B04A0903C0429
:1046C000B0903D049701A801B601C5010E945B0BA3
:1046D000982E0A191B0917FF03C01195019511099E
:1046E000EC18FD08F7FE03C0F194E194F108E00E28
:1046F000F11E8091560481111CC0992009F41DC13E
:10470000B1E0B0935604109255040E9496098FE1CF
:104710009AE00E94470A81E19AE090938304809393
:1047200082048AE58093810480915604882309F4E9
:1047300064C0992009F420C1109255048091380476
:10474000811104C08FE19AE00E94470A80913C04E5
:1047500090913D044091840450918504481B590B6D
:1047600060913A0470913B04209186043091870453
:10477000261B370B04E010E04131510544F410E0F2
:1047800000E0403FAFEF5A0714F40CEF1FEFE4E0F6
:10479000F0E02131310544F4F0E0E0E0203FBFEFEC
:1047A0003B0714F4ECEFFFEF7B01EE0EFF1E080F4A
:1047B000191F57FF03C051954195510937FF03C099
:1047C000319521953109241735070CF013C1C80123
:1047D0000E94940C811104C010933D0400933C048A
:1047E000B70180913C0490913D040E94940C81118A
:1047F00004C0F0923B04E0923A04809186049091C8
:104800008704209184043091850440913C045091A8
:104810003D04241B350B23593F4F2B3D310508F038
:10482000BFC020913A0430913B04821B930B835903
:104830009F4F8B3D910508F0B3C0109253040E9426
:10484000960985E00E947F0CABC088E129CE8730B5
:1048500009F45BC0883009F020CF40E0612F8F2D34
:104860000E940D0B8BE69BE00E94470A8AE899E0C4
:1048700090938304809382048AE5809381048091DD
:104880009C048F5F80939C0408CF40E0612F8F2DA4
:104890000E940D0B8BE69BE00E94470A8091510419
:1048A000833008F0FACE8F5F80935104813051F449
:1048B00080E899E090938304809382048AE5809352
:1048C0008104EBCE823019F486E799E0F3CFA1E0C2
:1048D000A093940489E599E0EDCF40E0612F8F2DFE
:1048E0000E940D0B8BE69BE00E94470A8BEC99E03F
:1048F00090938304809382048AE58093810480915D
:104900009D048F5F80939D04C8CE40E0612F8F2D62
:104910000E940D0B8BE69BE00E94470A8AEA99E011
:1049200090938304809382048AE58093810480912C
:104930009B048F5F80939B04B0CE80919104882369
:1049400009F45BCFE114ECE0FE060CF056CF0E94B8
:10495000140D8F719927892B09F04FCFF1E0F09357
:104960005604109255040E9496098FE19AE00E9425
:10497000470A8FEF99E0D1CE21E0E21625E0F2065A
:104980000CF4DACE809155048B3420F48F5F809341
:104990005504D4CE10925604109255040E949609E4
:1049A000809186049091870497FF02C081509F4FA9
:1049B000692F809184049091850497FF02C08150F3
:1049C0009F4F892F0E942B0B843061F480919404B7
:1049D000882339F1E1E0E09353040E94960985E0D1
:1049E0000E947F0C80919204811137CC0E9496091D
:1049F00085E074CCB7010E94940C811104C0F09240
:104A00003B04E0923A0460913A0470913B04C8017F
:104A10000E94940C8111F1CE10933D0400933C044C
:104A2000ECCE8091820490918304892BD9F685E99C
:104A30009AE090938304809382048AE580938104B2
:104A4000D1CF80915804909159048E31910528F46A
:104A50000196909359048093580480915804909142
:104A600059044E9709F0F9CB0E94E90A8111F5CB60
:104A700010E000E0F12CE12C4DE00BC00115110518
:104A8000D9F3F3E2EF16F104B9F30B311105A1F3F9
:104A900040E0602F8E2D0E940D0B2FEFE21AF20ADC
:104AA00034E2E316F10451F70F5F1F4F0C3111058B
:104AB00009F7E12C00E02AE142E261E081E00E9496
:104AC0002F0D10E0D12CC12CFF24F394E12C00E039
:104AD000B12C90E0B016E8F4A12C9F2C9B0C9923EC
:104AE00041F091E01AC091111BC0B12CF3CF81119C
:104AF0000EC06E2D6A0D892D0E942B0BA394A0125F
:104B0000F6CF91E0811101C090E0B394E3CF91E042
:104B1000FCCF911102C01017E8F10F5F0C3119F7AB
:104B2000E3944BE1E412D3CFF39453E2F512CECFEA
:104B30001730A0F102E0812F8250990B7C01F2E046
:104B40007F2E7D0CA2E08A2E8C0C8D2D810FBDEF67
:104B5000BB2EB80E1C0D13500E151F040CF0B1CF58
:104B6000902E9C0C4DE0672D892D0E940D0BA02EE0
:104B7000AD0C4DE06A2D882D0E940D0B4DE06B2D84
:104B8000892D0E940D0B4DE06A2D812F0E940D0B87
:104B90000F5FE2CF102FDE2CCF2CBFCF11E040E013
:104BA000612F81E00E940D0B40E0612F82E00E94A6
:104BB0000D0B40E0612F83E00E940D0B1F5F14304E
:104BC00071F776E2C72EE8E1EE2EF12C0E94140D6B
:104BD0008F71A82E02E0080F0E94140DB7010E94E9
:104BE0008C2DB82E62E0D62ED80E6D2D802F0E940F
:104BF0002B0B811132C06D2D83E08A0D0E942B0B8F
:104C000011E0811110E063E06B0D802F0E942B0BEF
:104C1000811101C01F5F6D2D81E08A0D0E942B0B59
:104C2000811101C01F5F61E06B0D802F0E942B0B73
:104C3000811101C01F5F133080F0AD2DA150BB0B5F
:104C4000E02FE150FF0BCF018A0F9B1F06972CF03E
:104C50004DE06D2D802F0E940D0BCA94C110B6CF70
:104C600040EBC42E44E0D42E53E0B52E0E94140D28
:104C700062E270E00E948C2D082FA82E8824839475
:104C8000880E0E94140D6AE170E00E948C2D182F8E
:104C9000982E77247394780E080F672D882D0E9424
:104CA0002B0B811147C0063008F444C032E0F32ECC
:104CB00001E0FA2DF11BF88B2F2D220F2A87EE240D
:104CC000E3943889310F3C875A2C501A4F2C490CE9
:104CD000392C301A2F2C2A0C652C6E0C612F862D46
:104CE0000E942B0B853021F1642D862D0E942B0B09
:104CF0008530F1F0632C6E0C662D8C850E942B0B99
:104D00008530B1F0662D822D0E942B0B853081F00D
:104D1000E3944A85E412E0CF0F5FF394115004321C
:104D200059F645E0672D882D0E940D0BBA9402C0FC
:104D30000730B8F751E0C51AD10811F0B11096CF7D
:104D400000E213E092E2E92EF12C2AE1C22ED12CEE
:104D50000E94140DB7010E948C2D782E99249394F3
:104D6000980E0E94140DB6010E948C2DA82E882446
:104D70008394880E682E670C682F892D0E94530B30
:104D8000BB24B394811101C0B12C682D82E0870D42
:104D90000E94530B8111B39462E06A0D892D0E9429
:104DA000530B8111B394682D872D0E94530B8111F1
:104DB000B394682D892D0E942B0B811105C08CE0C6
:104DC000861510F4B110B6C00150110909F0C0CF1A
:104DD000212C312C00E0B8E7CB2EB5E0DB2E12E21F
:104DE000812E912C8AE1682E712C0E94140DB40141
:104DF0000E948C2D182F55245394580E0E94140D88
:104E0000B3010E948C2D44244394480EA52CB12C50
:104E1000E42CF12C180F642D852D0E942B0B811191
:104E200016C00117A0F4173190F07E2D6627605848
:104E30007F4F9A2D882720E831E040E851E08058E4
:104E40009F4F0E945B0B811102C0012F120191E064
:104E5000C91AD10851F6002329F041E0622D832DB3
:104E60000E940D0B80E891E0909385048093840468
:104E7000909387048093860480E28093880484E67C
:104E80008093930410928F0410928E0410929004D9
:104E90001092910410928A041092890410928C044A
:104EA00010928B0410928D0410924F0410924E04B5
:104EB000109254041092560410925504109251040A
:104EC0001092940410E000E0612F802F0E942B0BC1
:104ED0008130B1F5202F30E0322F222720583F4F6C
:104EE00030933D0420933C04212F30E0322F2227C1
:104EF00020583F4F30933B0420933A04809354044E
:104F000040E0612F802F0E940D0B2FB7F894809105
:104F1000630490916404A0916504B09166042FBF6E
:104F200080935E0490935F04A0936004B093610447
:104F300082E0D4C944E0682D892D0E940D0B48CF32
:104F40000F5F043209F0C0CF1F5F1C3109F0BBCFE7
:104F5000DCCF0E94140D0E94E90A857031F0809127
:104F60005204857011F4109258040E94E90A8A7064
:104F700039F0809152048A7019F4A1E0A09358048A
:104F80000E94E90A807359F080915204807339F4C9
:104F900080915804882341F0813009F44AC00E946E
:104FA000E90A8093520459C9109251041092940452
:104FB0001092530484E08093950410929A04109206
:104FC0009D0410929B0410929C04109296041092DF
:104FD0009704109298041092990480E891E09093BD
:104FE000850480938404909387048093860480E2F0
:104FF0008093880484E68093930410928F04109227
:105000008E04109290041092910410928A041092CF
:10501000890410928C0410928B0410928D041092CB
:105020004F0410924E048093920481E00E947F0C02
:10503000B6CF80913E04811110C00E94640A11E035
:1050400090E080E00E94262D181709F4A8CF612F68
:1050500090E080E00E942E2DA2CF0E945F0A10E017
:10506000EFCF0E94E90A182F80910301882339F0BD
:10507000111102C01092030110935704EEC8812F42
:105080008F7059F0809157048F7039F481E09091BE
:105090005804911180E080935804812F807361F34C
:1050A00080915704807341F780915804811107C0A3
:1050B000B1E0B093030182E00E947F0CDDCFE1E01C
:1050C000E09303010E9496091092830410928204D7
:1050D00010928104109256041092550410925404B8
:1050E000109253041092580480E0E6CF8091580447
:1050F000909159044F9709F0B0C80E94E90A8111B4
:10510000ACC8ECC8823009F4C8C0B0F4882309F4F4
:1051100058C0813009F4B2C0EEE9F4E020E080E04C
:1051200098E000800EBC2111012C019780FDFDCF7D
:105130000192B9F70DB455C8843009F463C408F47A
:105140003EC4853049F78091580490915904892BC9
:1051500031F481E090E090935904809358040FEF6C
:1051600010E02091580430915904C9019695879513
:10517000909359048093580420FF08C0EEE68E27D0
:10518000EFE19E279093590480935804809158042E
:1051900090915904BC01660F672F661F770B7195BC
:1051A00077278F7740E090E00E94770A809158043B
:1051B00090915904019709F044C484E00E947F0C47
:1051C000ABCF0E940307EBEBF4E08491ECEBF4E04F
:1051D000E49190E00097C1F1EE23B1F12E2F2695D6
:1051E0002695269530E0E77011F02F5F3F4F6EE96E
:1051F000E62E64E0F62E10E000E070E060E0261796
:10520000370711F168307105F9F0D70150E040E03F
:10521000F801E354FB4F6F01F601E40FF51FF49121
:10522000EC91EF2BEC934F5F5F4F4817590724F435
:1052300011964038510581F76F5F7F4FF0E8EF0E10
:10524000F11C080F191FDBCF80913E0420E04CE6D3
:1052500066E0882381F088EB94E00E94F10C809155
:10526000580447E0811141E520E066E082EB94E0DC
:105270000E94F10C51CF84EB94E0EFCF0E94030722
:1052800021E04EE262E087EC98E00E94F10C21E020
:105290004EE264E08DEB98E0EBCFA0908404B090F8
:1052A0008504B0924004A0923F04C0908604D09040
:1052B0008704D0924204C092410490908804909256
:1052C0004304809134048F5F809334045EE9652E3B
:1052D00054E0752EF30190E02FEF892F837009F4CD
:1052E000DBC0823009F4DAC080E02193DF01A158ED
:1052F000BF4F2C93A058BF4F2C93A058BF4F2C9357
:10530000A058BF4F8C93A058BF4F8C93A058BF4F4D
:105310008C93A058BF4F8C939F5F9038F1F61092FA
:1053200033041092D60880914E0450914F04505E81
:10533000A3EBB3E0082E000C990B9C0146E0220F72
:10534000331F4A95E1F7E3E3F3E040E01D92652F58
:10535000630F61934F5F281B390B4038B9F7C501C4
:10536000B7FE02C081509F4F90934C04C601D7FEF8
:1053700002C081509F4F90934D04192D1195812F9C
:105380000E94DE1A7C019093450480934404E12F2F
:10539000F0E0EE0FFF1FE755F44F059114911093C5
:1053A00047040093460480E2882E8918882D0E94C5
:1053B000DE1A9093490480934804E82DF0E0EE0F44
:1053C000FF1FE755F44F8591949190934B04809380
:1053D0004A04892D0E94DE1AE92DF0E0EE0FFF1F2E
:1053E000E755F44F2591349167E0689FA001699FCC
:1053F000500D11244A0D5B1D629FC001639F900DEB
:1054000011248C0D9D1D38EFD32ED90E88EF850FFA
:1054100087FD80E0D7FCD12CC82E24E1281714F496
:10542000A4E1CA2E3CE03D1514F4FCE0DF2EE0E1DF
:105430009E2E9C0CBB24B3941E141F043CF0992494
:105440009A949C0C4FE0C40EBB24BA9470E1A72E32
:10545000AD0C8824839417FD07C0AA24AA94AD0C30
:105460005FE0D50E88248A94F7FE03C0F194E1949E
:10547000F10817FF03C0119501951109E016F10617
:1054800094F4AD14D9F01C2D911651F06D2D812F8F
:105490000E9456191B0DF8CF85E527CF8AEA25CF44
:1054A000D80CEFCFCB0C9C1449F01D2DA116D1F3D5
:1054B000612F8C2D0E945619180DF8CF009184048D
:1054C0001091850414500027E0908604F090870422
:1054D00084E0F81AEE24D12CC12C470198EF991AD8
:1054E0005801A8EFBA1AC8018C0D9D1D9401AC019A
:1054F000B7010E94D015B7016C0D7D1D9B01A50160
:10550000C8010E94D015BEEFDB1AC114EAE0DE0626
:1055100051F74090840450908504F4E05F1A4424CD
:10552000009186041091870414500027120127EF80
:10553000321A7201480138EF931A5801A418B508BD
:10554000620148EFD41A9401A701B801C7010E9473
:105550001115B5016E0D7F1D9B01A601C2010E94B0
:105560001115F3942E143F0471F78091540488238D
:1055700009F4CFC060913A0470913B049E012F5F03
:105580003F4FAE014A5F5F4F80913C0490913D04D4
:105590000E94BA13882309F4BCC0E980FA8022E68D
:1055A00030E0D7010E94BC2D20E830E040E050E020
:1055B0000E943C2D121613060CF0ABC01901220CF0
:1055C000331CC101032C000CAA0BBB0B8C879D87DD
:1055D000AE87BF8728E130E0D1010E94BC2D4B018E
:1055E0005C0164E0B594A794979487946A95D1F789
:1055F00064018E819F81910137FE02C02F5F3F4F72
:10560000359527952C01421A530A0E948E10082EB8
:10561000000C990BAFEFEA16F1040CF073C0B1E087
:10562000BE0DBA87E818F9085701A80EB91E720115
:10563000240C351C46018A0C9B1C9601DD0C440B86
:10564000550B288B398B4A8B5B8BE214F3040CF0DF
:1056500060C030E8E316F10408F057C0F701ED54DC
:10566000FC4F80814A85841708F04FC0B701641948
:105670007509072E000C880B990B24E0660F771F25
:10568000881F991F2A95D1F72C853D854E855F850A
:105690000E943C2D8501C22ED12C08151905ACF5B0
:1056A0000034110560F528E130E0D801AA19BB09E2
:1056B0000E94BC2D288939894A895B890E943C2D2A
:1056C000E22FF0E083E0F595E7958A95E1F794E025
:1056D000EE0FFF1F9A95E1F7EC0DFD1DEF52F74F0E
:1056E000E491F0E0277002C0F595E7952A95E2F77E
:1056F000E0FF05C040E0B801C7010E94770A0F5FD4
:105700001F4FCBCFEFEFEA878DCF5FEFE51AF50A9A
:105710009CCFB12C17E0A12E8091D608B81608F0C6
:10572000DAC0AB9CC0011124FC01E256F74F808027
:10573000918006812380228120FD58C08056974F9A
:10574000DC01CC90C1FACC24C0F82581148121342D
:1057500090F4B2E0EB2E213248F4822F90E0EE2458
:10576000E39441971CF4233040F0E12C412F622D4B
:10577000C4010E949C10B394CFCF822D022C000C48
:10578000990BFC01ED54FC4F7F018081223031F5F3
:10579000801778F4C22CD12C612F70E040E0C60154
:1057A0000E94770A61E0610F70E040E0C6010E944C
:1057B000770AD70111968C918017E8F62394312C43
:1057C000612F70E040E0C1010E94770A1F5F612FE6
:1057D00070E040E0C1010E94770ACDCF801758F6F3
:1057E000612F70E040E0822D90E0F5CFE02FF0E0F7
:1057F000FB87EA87022C000C3308EE0FFF1FFD87A2
:10580000EC87C1010E948E10D40114965C9050FA6E
:10581000552450F8F4013D96F98BE88B7401F5E0BE
:10582000EF0EF11C282F880F330B3D8B2C8B4889F2
:105830005989E416F50609F49ECFD7012C9120383A
:1058400009F445C04C855D8524036001259FD00C7B
:105850001124CD2CDD0CDD08C20CD31C11962C912B
:1058600024038001259F100D1124012F110F110B0E
:105870008C899D89080F191F9FE7C916D10438F537
:105880000F33110520F5F601ED54FC4F8081AA85F8
:10589000BB858A171B0609F0D4F4452DB801C60153
:1058A0000E94770A882483948C0C912C452DB80192
:1058B000C4010E94770A0F5F10E0452DB801C401B2
:1058C0000E94770A452DB801C6010E94770AB4E00C
:1058D000EB0EF11CACCF80918F048823F1F02CE10A
:1058E00035E0F30181818E7F8183EF57FC4F80810A
:1058F0008F778083FFEF6F1A7F0A2615370589F7A8
:10590000EEE9F4E01082DF01A158BF4F1C92E0588D
:10591000FF4F28E0EE39F207A9F720E042E567E003
:1059200084E099E00E94F10C8091510490E000978E
:1059300071F1FE01319610E000E02AE030E00F5FE7
:105940001F4FB9010E948C2D805D8193CB010530E2
:10595000110511F0009799F741E050E04C0F5D1FE1
:10596000040F151F44E8E42E48E0F42E01501109FD
:10597000888599858017910781F040E0D8016C9166
:10598000C7010E94D10CB4E0EB0EF11CEFCF40E058
:1059900060E384E898E00E94D10C20E04AE667E0EA
:1059A00081E099E00E94F10C80918204909183043F
:1059B00020E040E060E0009709F05ACCADCB0E94B7
:1059C000030721E044E361E089E199E00E94F10CE2
:1059D00021E04AE263E080E199E00E94F10C21E0DD
:1059E00048E365E08BE099E00E94F10C8091580457
:1059F00042E263E0882311F040E365E021E089E0C2
:105A000099E036CC0E9403078091530421E088235B
:105A100061F04AE262E08DE299E00E94F10C21E03F
:105A200046E264E080E299E023CC48E262E08CE464
:105A300099E00E94F10C21E048E164E089E399E0FB
:105A400017CC0150110909F08CCB66CBF999FECF28
:105A500092BD81BDF89A992780B50895262FF999AE
:105A6000FECF1FBA92BD81BD20BD0FB6F894FA9A41
:105A7000F99A0FBE01960895052E97FB1EF4009427
:105A80000E94532D57FD07D00E945B2D07FC03D0C9
:105A90004EF40C94532D50954095309521953F4FE1
:105AA0004F4F5F4F089590958095709561957F4F0A
:105AB0008F4F9F4F0895A1E21A2EAA1BBB1BFD0119
:105AC0000DC0AA1FBB1FEE1FFF1FA217B307E407DD
:105AD000F50720F0A21BB30BE40BF50B661F771F35
:105AE000881F991F1A9469F7609570958095909515
:105AF0009B01AC01BD01CF010895A29FB001B39FEE
:105B0000C001A39F700D811D1124911DB29F700DC6
:105B1000811D1124911D0895AA1BBB1B51E107C0D3
:105B2000AA1FBB1FA617B70710F0A61BB70B881F2D
:105B3000991F5A95A9F780959095BC01CD010895BC
:105B400097FB072E16F4009407D077FD09D00E942A
:105B50008C2D07FC05D03EF4909581959F4F0895BC
:105B6000709561957F4F08950E947D2D332312F427
:105B70008A1B9B0B0C94BE2D0E947D2DB7FF0895B0
:105B8000821B930B0895EE0FFF1F0590F491E02DFB
:065B90000994F894FFCF18
:105B960001001001FFFFFFFF00E100000000000010
:105BA60000C18081000000000000005F07FD088042
:0A5BB600077507C6078407A2070061
:00000001FF
